:0300000002407348
:0C40730078FFE4F6D8FD7581700240BAB9
:101CAC000A53746172743A20004950436F6E6E652A
:101CBC0063745245510A004950436F6E6E656374EC
:101CCC00003E432C562C43432CC0E4E0EFF2E5F0ED
:101CDC0020D1E8EDEAEEEC49500A003E432C4D4190
:101CEC00432C25303262583A25303262583A25302E
:101CFC003262583A25303262583A25303262583ABC
:101D0C0025303262582C4D414320E0E4F0E5F10AD5
:101D1C00003E432C5645522C20332E3120EEF2201F
:101D2C0025732025732CC2E5F0F1E8FF20495020E3
:101D3C00ECEEE4F3EBFF0A004170722030322032FB
:101D4C003030380031373A32323A3531003E432C9C
:101D5C004C442C50524F473A202020202020202049
:101D6C002020202020202020202020202020202067
:101D7C002020202020202020202020202020202057
:101D8C002020202020202020202020202020202047
:101D9C00202020202020202020202020202CC4E0C7
:101DAC00F2E020EFF0EEF8E8E2EAE828F4E0E9EB04
:101DBC00290A003E2A2C312CCEF1EDEEE2EDFBE5AA
:101DCC0020EFE0F0E0ECE5F2F0FB20F1E5F2E5E2EB
:101DDC00EEE3EE20E8EDF2E5F0F4E5E9F1E00A00DF
:101DEC003E412C4130312C2562752E2562752E25F5
:101DFC0062752E2562752C495020E0E4F0E5F12047
:101E0C00E0E4E0EFF2E5F0E00A003E412C41303234
:101E1C002C2562752E2562752E2562752E25627510
:101E2C002C495020E0E4F0E5F120EEF1ED2E20F10C
:101E3C00E5F0E2E5F0E00A003E412C4130332C2580
:101E4C0062752E2562752E2562752E2562752C49BC
:101E5C005020E0E4F0E5F120F0E5E72E20F1E5F08C
:101E6C00E2E5F0E00A003E412C4130342C2562754D
:101E7C002E2562752E2562752E2562752CCCE0F10F
:101E8C00EAE020F1E5F2E80A003E412C4130352C25
:101E9C002562752E2562752E2562752E2562752C90
:101EAC00D8EBFEE70A003E532C4130362C256275E8
:101EBC002CC2F0E5ECFF20EEE6E8E42E20EAE2E8A6
:101ECC00F2E0EDF6E8E820282A3130ECF1290A009E
:101EDC003E2A2C312CC4EEEF2E20EFE0F0E0ECE5A6
:101EEC00F2F0FB20F1E5F2E5E2EEE3EE20E8EDF2B4
:101EFC00E5F0F4E5E9F1E00A003E422C5330312CD8
:101F0C002562752CC6E4E0F2FC20E7E0EFF0EEF180
:101F1C00E020F1EEE5E4E8EDE5EDE8FF20EEF2205F
:101F2C00F1E5F0E2E5F0E00A003E422C5330322CB1
:101F3C002562752CCEE1ECE5ED20F120F1E5F0E227
:101F4C00E5F0EEEC20E1E5E720EAE2E8F2E0EDF680
:101F5C00E8E90A003E422C5330332C2562752CCF15
:101F6C00E5F0E5E7E0EFF3F1EA20EFF0E820EFEE43
:101F7C00F2E5F0E520F1E2FFE7E820F120F1E5F0F1
:101F8C00E2E5F0EEEC0A003E422C5330342C256294
:101F9C00752CCDE5F220EFE5F0E5E4E0F7E820E480
:101FAC00E8E0E3EDEEF1F2E8EAE820E220F1E5F01A
:101FBC00E2E5F00A003E422C5330352C2562752C9C
:101FCC00CAE0EDE0EB20F8E8F0EEEAEEE2E5F8E04E
:101FDC00F2E5EBFCEDEEE3EE20EEE1ECE5EDE00AF4
:101FEC00003E532C5330362C25303262582530327B
:101FFC0062582530326258253032625825303262B0
:10200C005825303262582C4D414320E0E4F0E5F184
:10201C0020F8E8F0EEEAEEE2E5F8E0F2E5EBFCEDB4
:10202C00EEE3EE20EEE1ECE5EDE00A003E454E4439
:10203C000A0044756D70582020202020303020304C
:10204C0031203032203033203034203035203036BF
:10205C002030372030382030392030412030422099
:10206C0030432030442030452030460A003A003AB4
:10207C0020000A0044756D70442020202020303050
:10208C002030312030322030332030342030352095
:10209C003036203037203038203039203041203055
:1020AC00422030432030442030452030460A004541
:1020BC007272206B657900526420656570726F6D69
:1020CC000A005264204D454D0A00526420436F644F
:1020DC00650A0044656275674950204F4E0A0044FA
:1020EC00656275674950204F46460A004465627523
:1020FC006755736572204F6E0A00446562756755AB
:10210C00736572204F46460A0044656275674D73CD
:10211C0067204F6E0A0044656275674D7367204FE8
:10212C0046460A00436F6E666967206C6F636B21CD
:10213C000A00577220656570726F6D0A002053613A
:10214C00766520656570726F6D210A00457272208C
:10215C004D414321004C6F61643E3E002A003C41DE
:10216C0030313D003C4130323D003C4130333D008C
:10217C003C4130343D003C4130353D003C41303633
:10218C003D003C21003C5330313D003C5330323D4E
:10219C00003C5330333D003C5330343D003C533015
:0921AC00353D003C5330363D0086
:0648EA00010B00010900B2
:1048D600C2AFC28E438910758BFF758DB7D2ABD22E
:0448E6008ED2AF229D
:03001B00023F455C
:103F4500C0E0C083C082C0D0C2AFC28E758BFF7582
:103F55008DB720060675A61E75A6E10509D202E5F0
:103F65000B6002050BE50AD394014002150A050E04
:103F7500E50E540F7050D20EE50E543F701AD20064
:103F850090668DE0601204F0E0D394B4400A90800E
:103F9500007480F0C2AF80FE906688E0600204F095
:103FA500906104E0600214F090668EE0D3940140C5
:103FB50003E014F0300502050CE50DD394644004CC
:103FC500D2068002050DE508D3940140021508D2FA
:0C3FD5008ED2AFD0D0D082D083D0E032AA
:10109600C291C290D2B5C20B7D027C007F07124876
:1010A6006A8F50E550646060097D017F60124802D6
:1010B600D20BE4FDFC7F0B12486A8F50E55030E6F8
:1010C600097D04E4FF124826D20B7D017C007F07D0
:1010D60012486A8F50E5507008FD7FFF124802D211
:1010E6000B300B03126000C2AFC288C2A8C2AA7539
:1010F6008900124388906341E0B4FA09A3E064CE04
:101106007003021196E4F55074392550F582E434E3
:1011160063F583E4F00550E550B443EC9063417405
:10112600FAF0A374CEF0A374CCF0906347740AF07F
:10113600E4A3F0A304F0A3F090634C7403F0A3744B
:10114600CCF090633D74FFF0A3F0A3F0E4A3F0901D
:1011560063587405F0E4F550E5502401FFE433FECE
:1011660074392550F582E43463F583E0FD1248BDF9
:101176000550E550C3944340DFE4F5A775A61E75F8
:10118600A6E1907FF0F0A3F09080007480F080FEDE
:10119600D2AF90634C7403F0A374CCF0E490634B2D
:1011A600F0123C77C2B5123EA7C20612468C906377
:1011B60058E0C3940350037403F0D20BC20DC20C63
:1011C600D293200B077E1C7FAC123988E490657899
:1011D600F01248D6C2AFA37408F09062B77424F038
:1011E600E4A3F0906341E09062B9F0906342E0902E
:1011F60062BAF0906343E09062BBF0906344E09083
:1012060062BCF0906345E09062BDF0906346E0906A
:1012160062BEF0750A01E490657AF0C207C208C2A0
:1012260009C20AD2AF75A70775A61E75A6E1200BDF
:1012360018AF50FE7D03123A89E4FF123D5D7E63CE
:101246007F78E4FB7D01123B8390668DE06003743A
:1012560001F0E4906104F0A37455F0A37481F0E406
:10126600F50CE4F50D906104E070031216DE90664D
:101276008EE0B401119080007410F0E490668EF058
:10128600D20BC20CC20D908008E0F55030E405D2B6
:10129600077410F0E55030E508D2099080087420F4
:1012A600F0E55030E608D2089080087440F0E50C6E
:1012B600D394034023908002E4F0908001F0908064
:1012C60000F0E50CD39406400FE4F50CC2039065DC
:1012D6007AF0750A0112468C9080A0E070031244E1
:1012E600069080B8E070031244809080D0E07003CE
:1012F60012456C908000E07013300710123884900D
:101306006334EFF0D394004003120026908002E08D
:101316007006908000E06005D205021268C205E4FE
:10132600F50C906104E06003021268300912123471
:10133600EC906334EFF0D394004005E0FF120022F6
:101346002008030214C7123208906334EFF07003CA
:10135600021268906378E054BF247F700302142A57
:101366001470030214022402600302145D200B07AA
:101376007E1C7FB5123988300F7920037690635032
:10138600E07006906354E0605B906684E0FF9063D3
:1013960050E0B50724906685E0FE906351E0B506FF
:1013A60018906686E0FE906352E0B5060C9066875C
:1013B600E0FE906353E06E602B906354E06F7033F1
:1013C600906685E0FF906355E0B50727906686E056
:1013D600FF906356E0B5071B906687E0FF90635762
:1013E600E0B5070F90657A7401F01248F3750A01AB
:1013F6000214C790668474FFF00214C790668DE0ED
:1014060060037401F090667CE0FF90637AE06F60A1
:10141600030214C790667CE004F0E4F50A90657850
:10142600F00214C73003030214C7906347E0700349
:101436000212681248F2D203E4F50A906578F09039
:10144600668804F0E490667BF0A3F0200B737E1CA4
:101456007FC3123988806A90668DE060037401F05C
:10146600300352906378E020E74B90637AE0FF9078
:10147600667BE0FE6F600D906683E07007EE146F8A
:10148600703F801390667BE004F0906334E0FFD3F6
:101496009404400312484A9060007482F0A37401D9
:1014A600F090637AE0906002F07E607F007D031228
:1014B6004288021268300F0920030690668474FF82
:1014C600F02003030215A3E50A706B123652EF6093
:1014D600207E647F78906479E02404FD124288902F
:1014E6006683E06003021268906358E0F50A021210
:1014F60068906688E0D3943C403C906683E0703602
:1015060090668804F09062B6E0702B1248F1E49081
:101516006478F0A37412F090667CE090647AF0A38D
:1015260074FDF090610763A20190647C63A2017F61
:1015360012122DBE809B12001E8F50E550B401156D
:101546009060007483F0E4A3F07E607F007D021259
:101556004288021268E550D39401401C90600074E2
:1015660083F0A37401F0E55024FEA3F07E607F00B3
:101576007D03124288021268E50A640160030212C2
:1015860068906578E004F0E0C3940550030214D730
:10159600C203E490657AF01248F3021268E50A6421
:1015A60001600302126890657AE014604624FE60CA
:1015B6004214700302169124046003021268E4F5D3
:1015C6000C200F1390657A7404F0906578E054014E
:1015D600F0750A010212689080027410F0E49065BA
:1015E6007AF090657804F0750AC890668474FFF006
:1015F600021268906684E070030216809064787424
:1016060080F090647A7401F0E4A3F0A304F0A3746C
:1016160030F0A3747BF0E4F550747F2550F582E436
:101626003464F583747DF074802550F582E4346467
:10163600F583E4F0E5502407906479F07C667D84B8
:1016460090634CE0FAA3E0FB7F021241847E647F44
:1016560078E5502409FD124288906683E0601B12EB
:1016660048F2D203E4F50A906578F090668804F0B3
:10167600E490667BF0A3F002126890657A7404F039
:10168600906358E02432F50A0212689080027410C2
:10169600F0750A03906578E06401FFF090657A744E
:1016A60001F0EF7019906354E06013FCA3E0FDA312
:1016B600E0FEA3E0FF906684122BDB0212689063C3
:1016C60050E0FCA3E0FDA3E0FEA3E0FF90668412D9
:0716D6002BDB02126880FE0D
:0116DD0022EA
:10002600906379E0B444047F0180027F0090637896
:10003600E0B447047E0180027E00EE5F604A906372
:1000460041E090637AF0906342E090637BF09063C6
:1000560043E090637CF0906344E090637DF09063AE
:1000660045E090637EF0906346E090637FF0906396
:10007600797452F09062B063A2019080A863A201E5
:100086007F06122DBE02089A906334E0C39408508E
:10009600030208A3906341E0FF90637AE06F600378
:1000A6000208A3906342E0FF90637BE06F60030267
:1000B60008A3906343E0FF90637CE06F600302084F
:1000C600A3906344E0FF90637DE06F60030208A3A2
:1000D600906345E0FF90637EE06F60030208A390A3
:1000E6006346E0FF90637FE06F60030208A39063BE
:1000F60079E0B444159062B0E0B4FF0E63A20190BB
:1001060080A863A2017F06122DBE90668DE0600373
:100116007401F090668E7464F09063797452F09076
:100126006378E0646D60030202A37BFF7A1C79CDDD
:100136001226EE7BFF7A1C79E7906341E0F559A31E
:10014600E0F55AA3E0F55BA3E0F55CA3E0F55DA35B
:10015600E0F55E1226EE7559FF755A1D755B4475FE
:100166005CFF755D1D755E507BFF7A1D791D12263D
:10017600EE7BFF7A1D79591226EE7BFF7A1D79BF39
:100186001226EE7BFF7A1D79EC906347E0F559A3C2
:10019600E0F55AA3E0F55BA3E0F55C1226EE7BFFE3
:1001A6007A1E7916906350E0F559A3E0F55AA3E05C
:1001B600F55BA3E0F55C1226EE7BFF7A1E79449090
:1001C6006354E0F559A3E0F55AA3E0F55BA3E0F527
:1001D6005C1226EE7BFF7A1E797290633DE0F5593C
:1001E600A3E0F55AA3E0F55BA3E0F55C1226EE7BEF
:1001F600FF7A1E7995906339E0F559A3E0F55AA385
:10020600E0F55BA3E0F55C1226EE7BFF7A1E79B281
:10021600906358E0F5591226EE7BFF7A1E79DC12C0
:1002260026EE7BFF7A1F7905A20FE433F5591226D5
:10023600EE7BFF7A1F7935906683E0F5591226EE3C
:100246007BFF7A1F796090668DE0F5591226EE7B6A
:10025600FF7A1F79939062B6E0F5591226EE7BFF7E
:100266007A1F79C1A201E433F5591226EE7BFF7A93
:100276001F79ED90667DE0F559A3E0F55AA3E0F508
:100286005BA3E0F55CA3E0F55DA3E0F55E1226EE68
:1002960012337D7BFF7A2079381226EE229063781E
:1002A600E0644C70757E207F3E123988906380E052
:1002B600F551A3E0F552E4F5547E207F7912398892
:1002C6007D03AF52AE51123A897E207F7B12398868
:1002D600E4F553855282855183E0FF74822553F5F8
:1002E60082E43463F583EFF00552E552700205515E
:1002F6000553E553B410DC7E637F82E4FB7D101268
:100306003B837E207F7E1239880554E554C39410C2
:1003160040A77E207F7E12398822906378E0646C45
:10032600705CF5557E207F80123988E4F554AF5510
:100336007E007D03123A897E207F7B123988E4F5A0
:1003460053A855E6FF74822553F582E43463F5839A
:10035600EFF005550553E553B410E67E637F82E45E
:10036600FB7D10123B837E207F7E1239880554E583
:1003760054C3940840B87E207F7E12398822906349
:1003860078E0644B7061F553746A2553F582E43462
:1003960063F583E06032746A2553F582E43463F5CD
:1003A60083E0F46023746A2553F582E43463F583AD
:1003B600E0FF74802553F582E43463F583E0B507E6
:1003C600100553E553B408C09061047432F0020876
:1003D6009A9063787421F0300B0302089A7E207F8E
:1003E600BB12398802089A906378E0B4521A200B3F
:1003F600077E207FC31239889063787472F07E631B
:100406007F787D0812420822906378E0644970453F
:10041600200B077E207FCE123988906380E0F5514D
:10042600A3E0F552E4F553855282855183E0FF74CB
:10043600822553F582E43463F583EFF00552E552E5
:10044600700205510553E553B480DC7E637F787DE9
:100456008A12420822906378E064437079A3E064CC
:10046600527046200B077E207FD612398890638013
:10047600E0F551A3E0F552E4F553855282855183A8
:10048600E493FF74822553F582E43463F583EFF039
:100496000552E552700205510553E553B480DB7EE3
:1004A600637F787D8A12420822906379E064576000
:1004B600030208A3906380E0F551A3E0F55274822D
:1004C6002553F582E43463AD82FC7B80AF52AE5196
:1004D6001247A802089A906378E064446003020514
:1004E6006D906380E0FF6444700302089AEFB431B4
:1004F6000CC20B7E207FDF12398802089A90638037
:10050600E0B4300CD20B7E207FEB12398802089AB9
:10051600906380E0B4320CD20C7E207FF8123988CA
:1005260002089A906380E0B4330CC20C7E217F06E9
:1005360012398802089A906380E0B4340CD20D7E9A
:10054600217F1512398802089A906380E0B4350C31
:10055600C20D7E217F2212398802089A906380E0BC
:10056600FF12002102089A906104E07013200B0725
:100576007E217F301239889063787421F002089AC0
:100586009061047432F0906378E0FFB4510A908071
:10059600007480F0C2AF80FEEF64577045200B07F1
:1005A6007E217F3E123988906381E0906334F0E4C7
:1005B600F553906334E0FFE553C39F400302089A66
:1005C60074822553F582E43463F583E0FF906380FB
:1005D600E0255324AFF582E43461F583EFF005534B
:1005E60080D0906378E06453600302069C200B077A
:1005F6007E217F49123988906341E0FF9061B8E01F
:100606006F703C906342E0FF9061B9E06F7030908C
:100616006343E0FF9061BAE0B50724906344E0FFCE
:100626009061BBE0B50718906345E0FF9061BCE0C0
:10063600B5070C906346E0FF9061BDE06F601690D1
:1006460063787421F0300B0302089A7E217F5812DA
:10065600398802089AE4F553E4F50DAF53FE74AFFA
:100666002553F582E43461F583E0FD1248BD055358
:10067600E553C394FE40E19080007480F0C2AFE47D
:10068600907FF0F0A3F0907FFD74AAF0A374FFF0C2
:10069600A37455F080FE906378E0644F704C9063CD
:1006A60080E0F551A3E0F552E5524551700A200B62
:1006B600077E217F61123988200B077E217F681211
:1006C6003988E4F55374822553F582E43463F5835F
:1006D600E0855282855183F00552E552700205513C
:1006E6000553E553B480DE02089A906378E0FFB4C0
:1006F60045279080007480F0906380E0FDA3E09031
:100706007FF0CDF0A3EDF0C2AF907FFD74AAF0A309
:1007160074FFF0A37455F080FEEF64656003020871
:100726009A906380E0FFA3E0907FF0CFF0A3EFF014
:10073600E4F551F552D3907FF1E09552907FF0E0C9
:1007460095514020E4F50D2552FFE5513401FE8513
:100756005282855183E0FD1248BD0552E552700272
:10076600055180D17E217F6A1240FFEF4E60201234
:100776000003906347EFF0120003906348EFF01216
:100786000003906349EFF012000390634AEFF07E96
:10079600217F701240FFEF4E6020120003906350DD
:1007A600EFF0120003906351EFF0120003906352D2
:1007B600EFF0120003906353EFF07E217F76124034
:1007C600FFEF4E6020120003906354EFF012000317
:1007D600906355EFF0120003906356EFF01200039A
:1007E600906357EFF07E217F7C1240FFEF4E602032
:1007F60012000390633DEFF012000390633EEFF0AA
:1008060012000390633FEFF0120003906340EFF095
:100816007E217F821240FFEF4E602012000390631C
:1008260039EFF012000390633AEFF0120003906381
:100836003BEFF012000390633CEFF07E217F8812BD
:1008460040FFEF4E600812462F906358EFF0E4F534
:1008560053E4F50DE5532401FFE433FE74392553C3
:10086600F582E43463F583E0FD1248BD0553E55394
:10087600C3944340DC9080007480F0C2AFE4907F64
:10088600F0F0A3F0907FFD74AAF0A374FFF0A374B8
:0D08960055F080FE7E637F787D08124208D9
:0108A3002232
:10477000AE07EEC39430400BEED394395005EE24CF
:10478000D0FF22EEC39461400BEED394665005EE49
:1047900024A9FF22EEC39441400BEED3944650056A
:0847A000EE24C9FF22AF06223E
:1048A3009062AFE004F070069062AEE004F09062B4
:0A48B300AEE0FEA3E0FF12488722EA
:100003001248A3124770EFC454F0FEC0061248A36F
:08001300124770D0E02FFF221C
:10462F00E4906BA9F01248A3906BAAEFF0C39430FB
:10463F004018E0FFD394395011906BA9E02407F58F
:10464F0082E43461F583EFF08011906BA9E02407C9
:10465F00F582E43461F583E4F0800C906BA9E004FB
:10466F00F0E0D3940840BE755900755A00755B0091
:0C467F00E4F55C7B017A617907122ECC17
:01468B00220C
:0440FF008E568F57F3
:104103009062AEE4F0A374FFF01248A3EF606EF484
:10411300606B855782855683E493B507EC75580128
:10412300E5572558F582E43556F583E493602590E9
:1041330062AFE02558FF9062AEE03400FE1248877C
:10414300E5572558F582E43556F583E493B507041E
:10415300055880CCE5572558F582E43556F583E4B8
:104163009370A6E55824FFFFE434FFFE9062AFE0AE
:104173002FF09062AEE03EF07E007F0122E4FEFF6E
:014183002219
:103C77007E217F8E1240FFEF4E70037F01227E214F
:103C87007F911240FFEF4E600C1248A3EF24D0241F
:103C9700FF920F8002D20F7E217F971240FFEF4ED7
:103CA700600C1248A3EF24D0906683F08005E4905F
:103CB7006683F07E217F9D1240FFEF4E600C124815
:103CC700A3EF24D090668DF08005E490668DF07E9A
:103CD700217FA31240FFEF4E600C1248A3EF24D0C0
:103CE7009062B6F08005E49062B6F07E217FA9125B
:103CF70040FFEF4E600C1248A3EF24D024FF92013F
:103D07008002C20190634163A20190667D63A201B4
:103D17007F06122DBE30013B7E217FAF1240FFEFA1
:103D27004E603012000390667DEFF012000390663C
:103D37007EEFF012000390667FEFF01200039066AB
:103D470080EFF0120003906681EFF0120003906697
:063D570082EFF07F002264
:1046E500906579E0C3947C503D906579E0FE04F0D7
:1046F50074B72EF582E43462F583EFF0BF0A279094
:104705006579E0FF04F074B72FF582E43462F58330
:10471500E4F0906579E0FF123E079065797408F042
:074725009062B8E004F022ED
:10468C009080007480F090633963A201F583F58209
:10469C0063A2017F08122DBE90634163A20190803A
:1046AC008863A2017F0A122DBE908092E4F0A3745D
:1046BC0032F0A37401F090634BE0FF9080B1F09066
:1046CC0080E1EFF09080957455F0A3F09080007429
:0946DC0001F090800974F0F02255
:10440600908009E04410F09080A0E0706C9080A14C
:104416007482F09080A874FFF0A3F0A3F0A3F07F5D
:10442600039080AEEFF07FCBA3EFF07F039080ACDC
:10443600EFF0A374CBF09080007402F0906B9D12A5
:104446002BE700000000906B9DE0908040F0906BA1
:104456009EE0908041F0906B9FE0908042F0906BE0
:10446600A0E0908043F0A3E4F0A3F0A3F0A3F090C3
:094476008018F0A3F0A3F0A3F0FC
:01447F00221A
:10456C00908009E04440F09080D17482F090634CCC
:10457C00E0FF9080DEF090634DE0FF9080DFF090E4
:10458C0080027402F0906BA1122BE70000000090E7
:10459C006BA1E0908058F0906BA2E0908059F09065
:1045AC006BA3E090805AF0906BA4E090805BF0A33A
:1045BC00E4F0A3F0A3F0A3F0908030F0A3F0A3F00C
:0245CC00A3F05A
:0145CE0022CA
:10448000908009E04420F09080B8E0706C9080B992
:104490007482F07F039080C6EFF07FCDA3EFF07FB2
:1044A000039080C4EFF0A374CDF09080C074FFF04F
:1044B000A3F0A3F0A3F09080017402F0906BA5121A
:1044C0002BE700000000906BA5E090804CF0906B13
:1044D000A6E090804DF0906BA7E090804EF0906B3E
:1044E000A8E090804FF0A3E4F0A3F0A3F0A3F09035
:0944F0008024F0A3F0A3F0A3F076
:0144F90022A0
:104184008C518D52A907EAFDE975F018A424ACFFFF
:10419400E5F034808F82F583EDF0EBFDE975F018DE
:1041A400A4FFAEF024ACFBEE34808B82F583A3ED48
:1041B400F08552828C83E0FDEF24A8FFEE3480FE6C
:1041C4008F82F583EDF08552828C83A3E08F828EFB
:1041D40083A3F0855282855183A3A3E0FDE975F0A2
:1041E40018A424A8FFE5F03480FE8F82F583A3A3EE
:1041F400EDF08552828C83A3A3A3E08F828E83A3E8
:04420400A3A3F0225E
:064208008D56AB07AA066B
:10420E00908000E020E572906B9DE0FCA3E0FDA3A2
:10421E00E0FEA3E0F55A8E598D588C57AE02AF03CF
:10422E008E838F8263A201E559540744C0F58385BE
:10423E005A8263A201AF56122E30E4FCFDFEE55AFF
:10424E002556F55AEE3559F559ED3558F558EC35E4
:10425E0057F557908040E557F0A3E558F0A3E55980
:10426E00F0A3E55AF09080007420F0AF5AAE59AD2D
:09427E0058AC57906B9D122BDB2C
:014287002214
:064288008D51AB07AA06F0
:10428E00908002E020E572906BA1E0FCA3E0FDA31C
:10429E00E0FEA3E0F5558E548D538C52AE02AF0363
:1042AE008E838F8263A201E554540744D0F5838533
:1042BE00558263A201AF51122E30E4FCFDFEE5558E
:1042CE002551F555EE3554F554ED3553F553EC3582
:1042DE0052F552908058E552F0A3E553F0A3E55401
:1042EE00F0A3E555F09080027420F0AF55AE54ADBA
:0942FE0053AC52906BA1122BDBB2
:014307002293
:023D5D008F5184
:103D5F00908001E030E5037F0022906BA5E0FCA38B
:103D6F00E0FDA3E0FEA3E0F5558E548D538C5290E9
:103D7F00667D63A201E554540744C8F583855582D7
:103D8F0063A2017F06122E46E5552406F555E4354C
:103D9F0054F554E43553F553E43552F55290657BA1
:103DAF0063A201E554540744C8F58385558263A285
:103DBF0001AF51122E46E4FCFDFEE5552551F55598
:103DCF00EE3554F554ED3553F553EC3552F552901D
:103DDF00804CE552F0A3E553F0A3E554F0A3E5556D
:103DEF00F09080017420F0AF55AE54AD53AC5290AB
:073DFF006BA5122BDBAF5195
:013E06002299
:103884009081E0E0F551055105510551055105516F
:1038940005510551055105510551908010E0F5542D
:1038A400A3E0F555A3E0F556A3E0F5579081E1E0D8
:1038B400F551055105510551055105510551055164
:1038C400055105510551908014E0F558A3E0F559D0
:1038D400A3E0F55AA3E0F55BE55AB55608E55BB5F8
:1038E40057037F0022E4F551E55A540744E0F58379
:1038F400855B8263A20190637863A2017F08122E24
:103904007690637A63A2019062B063A2017F06128B
:103914002DBE906378E0F552A3E0F553E4F55190A1
:103924006378E0702AA3E024F8F551E55A5407447B
:10393400E0F583855B8274082582F582E43583F59E
:103944008363A20190637863A201AF51122E76AE15
:1039540052E4FCFDE55B2553F55BE55A3EF55AED73
:103964003559F559EC3558F558908014E558F0A3BD
:10397400E559F0A3E55AF0A3E55BF09080007440AC
:03398400F0AF5150
:01398700221D
:103208009081E6E0F55105510551055105510551EB
:1032180005510551055105510551908028E0F55497
:10322800A3E0F555A3E0F556A3E0F5579081E7E054
:10323800F5510551055105510551055105510551E6
:1032480005510551055190802CE0F558A3E0F5593A
:10325800A3E0F55AA3E0F55BE4F551E55AB5560A43
:10326800E55BB55705C208023362E55A540744F0D6
:10327800F583855B8263A20190637863A2017F086E
:10328800122E76906378E0F552A3E0F553E55345A6
:103298005270099080027410F07F0022906684E0DA
:1032A800FFF4602D90637AE06F7076906685E0FF9A
:1032B80090637BE06F706A906686E0FF90637CE0C5
:1032C8006F705E906687E0FF90637DE06F6022809C
:1032D8005090637AE0906684F090637BE090668516
:1032E800F090637CE0906686F090637DE09066875E
:1032F800F0906378E0702AA3E024F8F551E55A5479
:103308000744F0F583855B8274082582F582E435ED
:1033180083F58363A20190637863A201AF51122EF3
:1033280076AE52E4FCFDE55B2553F55BE55A3EF5C8
:103338005AED3559F559EC3558F558AF57AE56ADE5
:1033480055AC54AB5BAA5AA959A858D3122BB7400D
:10335800099080027410F07F002290802CE558F0CC
:10336800A3E559F0A3E55AF0A3E55BF09080027459
:0433780040F0AF5121
:01337C00222E
:1034EC009081E3E0F5510551055105510551055108
:1034FC000551055105510551055190801CE0F554BD
:10350C00A3E0F555A3E0F556A3E0F5579081E4E070
:10351C00F5510551055105510551055105510551FF
:10352C00055105510551908020E0F558A3E0F5595F
:10353C00A3E0F55AA3E0F55BE4F551E55AB5560A5C
:10354C00E55BB55705C209023637E55A540744E81E
:10355C00F583855B8263A20190600463A2017F0EF8
:10356C00122E8C906004E0F552A3E0F55390600CA1
:10357C00E0FFF4604590667DE0FEEF6E706EA3E0B8
:10358C00FF90600DE06F706490667FE0FF90600EBE
:10359C00E06F7058906680E0FF90600FE06F704CA9
:1035AC00906681E0FF906010E06F7040906682E062
:1035BC00FF906011E06F60048032D2D9906004E01B
:1035CC00702AA3E024F2F551E55A540744E8F58338
:1035DC00855B82740E2582F582E43583F58363A2C4
:1035EC000190600463A201AF51122E8CAE52E4FC28
:1035FC00FDE55B2553F55BE55A3EF55AED3559F57E
:10360C0059EC3558F558AF57AE56AD55AC54AB5B7D
:10361C00AA5AA959A858D3122BB75006E5534552AC
:10362C0070099080017410F07F0022908020E55882
:10363C00F0A3E559F0A3E55AF0A3E55BF090800107
:05364C007440F0AF51D5
:013651002256
:043988008E568F5771
:10398C00E4F558F559908000E030E5110559E559FA
:10399C0070020558D39488E558941340E890800041
:1039AC00E030E503023A88906B9DE0FCA3E0FDA3B8
:1039BC00E0FEA3E0F55D8E5C8D5B8C5AE55DFFE56A
:1039CC005C5407FEE42FF559EE34C0F55885598246
:1039DC00F5837423F00559E559700205585358C7FF
:1039EC00F582855883740AF00559E559700205581B
:1039FC005358C790634163A20185588385598263EC
:103A0C00A2017F06122E3074062559F559E435585B
:103A1C00F55885568385578263A20185588385594D
:103A2C008263A201122E14E4FCFDFE906B9DE0F863
:103A3C00A3E0F9A3E0FAA3E02FFFEE3AFEED39FD87
:103A4C00EC38FCEF2408FFE43EFEE43DFDE43CFCD6
:103A5C00906B9D122BDB906B9DE0908040F0906BF7
:103A6C009EE0908041F0906B9FE0908042F0906BD4
:0C3A7C00A0E0908043F09080007420F0E7
:013A8800221B
:063B83008E568F578D588D
:103B8900E4F559F55A908000E030E511055AE55AF7
:103B990070020559D39488E559941340E890800040
:103BA900E030E503023C76906B9DE0FCA3E0FDA3C9
:103BB900E0FEA3E0F55E8E5D8D5C8C5BE55EFFE566
:103BC9005D5407FEE42FF55AEE34C0F559855A8243
:103BD900F5837423F0055AE55A700205595359C7FC
:103BE900F582855983EBF0055AE55A700205595358
:103BF90059C790634163A201855983855A8263A29B
:103C0900017F06122E307406255AF55AE43559F506
:103C19005985568385578263A201855983855A82BE
:103C290063A201AF58122E3074082558F558FFE4E5
:103C3900FCFDFEE55E2FF55EEE355DF55DED355C6F
:103C4900F55CEC355BF55B908040E55BF0A3E55CEA
:103C5900F0A3E55DF0A3E55EF09080007420F0AF7D
:0D3C69005EAE5DAD5CAC5B906B9D122BDB25
:013C7600222B
:023E07008F6AC0
:103E0900E4F56BF56C908000E030E511056CE56C2C
:103E19007002056BD39488E56B941340E890800099
:103E2900E020E579906B9DE0FCA3E0FDA3E0FEA313
:103E3900E0F5708E6F8D6E8C6DE570FFE56F540740
:103E4900FEE42FF56CEE34C0F56B9062B763A20106
:103E5900856B83856C8263A201AF6A122E30E4FC04
:103E6900FDFEE570256AF570EE356FF56FED356E7F
:103E7900F56EEC356DF56D908040E56DF0A3E56E5E
:103E8900F0A3E56FF0A3E570F09080007420F0AF27
:0D3E990070AE6FAD6EAC6D906B9D122BDBAB
:013EA60022F9
:063A89008E568F57AB05BD
:103A8F00E4F558F559908000E030E5110559E559F6
:103A9F0070020558D39488E558941340E89080003D
:103AAF00E030E503023B82906B9DE0FCA3E0FDA3B9
:103ABF00E0FEA3E0F55D8E5C8D5B8C5AE55DFFE566
:103ACF005C5407FEE42FF559EE34C0F55885598242
:103ADF00F5837423F00559E559700205585358C7FB
:103AEF00F582855883EBF00559E55970020558901A
:103AFF00634163A20185588385598263A2017F06C2
:103B0F00122E3074062559F559E43558F558535887
:103B1F00C7E556855982855883F00559E5597002D6
:103B2F0005585358C7F582855883E557F00559E571
:103B3F0059700205585358C7E55D240AF55DE43501
:103B4F005CF55CE4355BF55BE4355AF55A908040E3
:103B5F00E55AF0A3E55BF0A3E55CF0A3E55DF0901B
:103B6F0080007420F0AF5DAE5CAD5BAC5A906B9D86
:033B7F00122BDB2B
:013B82002220
:10488700E5D220E0FBC2AF438E2075D2028F828E25
:0B48970083E0FFE4F5D2538EDFD2AFC8
:0148A20022F3
:1048BD00E5D220E0FBC2AF43D2028F828E83EDF0B2
:0948CD0075D25063D250D2AF2223
:10438800E4FDED2401FFE433FE12488774392DF56E
:1043980082E43463F583EFF00DBD3FE6E4FDED24E0
:1043A8007FFFE433FE124887742F2DF582E43461D1
:1043B800F583EFF0742F2DF582E43461F583E07016
:1043C8001B742F2DF582E43461F5837420F074306A
:1043D8002DF582E43461F583E4F080040DBD80BEE0
:1043E800E49061AEF0FDEDFF7E0012488774AF2DBA
:0D43F800F582E43461F583EFF00DBDFEE9C0
:014405002294
:0247A8008B562E
:1047AA00A2AF9210C2AF85A25753A2FE8E838F8208
:1047BA0005A28C838D827409122EBAE55653A2FE85
:1047CA0043A220122EBC53A2DF8557A2A21092AF99
:0147DA00FFDF
:0147DB0022BB
:10486A00A2AF9210C2AF8C838D82EF122EBA43A2EE
:0C487A0020122EBC53A2DFA21092AFFF50
:01488600220F
:024802008F51D4
:10480400A2AF9210C2AFE4F5838D827406122EBA61
:10481400E55143A220122EBC53A2DFA21092AF7F17
:014824000192
:014825002270
:024826008F51B0
:10482800A2AF9210C2AFE4F5838D82740A122EBA39
:10483800E55143A220122EBC53A2DFA21092AF7FF3
:01484800016E
:01484900224C
:102CE300A907E7FFA805EF93C3966008403B74FC70
:102CF3002FFF80F00F08EF93C3966008402B74FBFF
:102D03002FFF80E00F08EF93C3966008401B74FA0F
:102D13002FFF80D00F08EF93D3966008400B74F910
:102D23002FFF80C01F1F1F1F1FEF54FEF80303F761
:102D3300E893FC08E893FD08E893FE08E893FF2274
:102D430009E993C39D6008402974FB29F980F109BF
:102D5300E993C39E6008401A74FA29F980E209E9ED
:102D630093D39F6008400B74F929F980D31919197B
:102D73001919E9C313C313FF22740093F8ECC39822
:102D83004024701F740193F8EDC3984019701474B4
:0E2D93000293F8EEC398400E7009740393F893
:102DA100EFC39840037F00227F0122EDF8E6F0088F
:102DB100A3DFFA22EDF8E0F608A3DFFA22E0A3632D
:102DC100A201F0A363A201DFF475A2002263A201B4
:102DD100F0A363A20122E0A363A201F0A363A20115
:102DE100E0A363A201F0A363A201E463A201F0A343
:102DF10063A201DFE175A20022E0A363A2016DFEDF
:102E0100936CFDEE058393FC158363A201DFEA75E4
:102E1100A200227F00E493A363A201F00F600CA340
:102E2100E583C2E3F58363A20180EA75A20022E093
:102E3100A363A201F0A3E583C2E3F58363A201DFEB
:102E4100EE75A20022E0A363A201F0A3E583C2E430
:102E5100D2E3F58363A201DFEC75A20022E0A36354
:102E6100A201F0A3E58344F8C2E5F58363A201DF83
:102E7100EC75A20022E583C2E3F583E0A363A2011E
:102E8100F0A363A201DFEE75A20022E583C2E4D2C2
:0A2E9100E3F583E0A363A201F0A3C0
:102E9B0063A201DFEC75A20022E58344F8F583E021
:102EAB00A363A201F0A363A201DFEE75A20022F9D6
:102EBB0022C002C004C00612FFF0D006D004D0021C
:012ECB0022E4
:1021B5003E2A2C312CCFE0F0E0ECE5F2F0FB20F8E4
:1021C500E8EDFB2043414E0A003E4C2C6B30312C90
:1021D50025732C43EAEEF0EEF1F2FC20EDE020F859
:1021E500E8EDE52043414E2C30202D20353030EAF6
:1021F500E1283530EC292C31202D203530EAE12835
:10220500353030EC290A0030202D20353030EAE118
:10221500283530EC290031202D203530EAE12835EC
:102225003030EC29003E2A2C312CCFE0F0E0ECE5F3
:10223500F2F0FB20EFF0EEF2EEEAEEEBE020D1DD7E
:10224500D22D34D2CC28CCE5F0EAF3F0E8E93233EC
:1022550030290A003E422C4930322C2562752CD299
:10226500E8EF20EFF0EEF2EEEAEEEBE020CCE5F061
:10227500EAF3F0E8E90A003E532C4930332C257384
:102285002CCFE0F0EEEBFC20E4EEF1F2F3EFE00A08
:10229500003E4C2C4930312C256C752CD1EAEEF0E2
:1022A500EEF1F2FC20EEE1ECE5EDE02C31323030E0
:1022B5002C323430302C343830302C393630302C08
:1022C50031393230300A003E422C4930352C2562F6
:1022D500752CCAEEEDF2F0EEEBFC20EFEE20EDE50D
:1022E500F7E5F2EDEEF1F2E80A003E532C49313202
:1022F5002C2562752CC0E4F0E5F120E1EBEEEAE077
:1023050020D2C8D220EDE020F8E8EDE50A003E53E2
:102315002C6D2562752C25732CCFF0E8E1EEF020AD
:102325002562752028C0E4F0E5F120E820EFE0F013
:10233500E0ECE5F2F0FB290A003E532C5630382C30
:1023450025752CCFE0F3E7E020E220EEEFF0EEF18B
:10235500E0F528ECF1290A003C21003C6B30313DC9
:10236500003C4930333D003C4930313D003C49316A
:10237500323D003C5630383D003C4930323D003C52
:102385004930353D002043616E4572474954002070
:102395000A002043616E457272434821000A000A13
:1023A500CEF2EAF0FBF2FC3A000A4669783A000AF6
:1023B500C7E0EFF0EEF13A00CFF0E8E5EC3A00CEF9
:1023C500F8E8E1EAE020CAD1210A00CED8C8C1CA9E
:1023D500C020C0E4F0E5F1E02100CED8C8C1CAC0F4
:1023E50020EEF2EAF0FBF2E8FF20EAE0EDE0EBE0B8
:1023F5002100204F4B212000CED8C8C1CAC020E7FC
:10240500E0EFF0EEF1E00000C1814001C080410144
:10241500C0804100C1814001C0804100C1814000B0
:10242500C1814001C0804101C0804100C18140009F
:10243500C1814001C0804100C1814001C08041018E
:10244500C0804100C1814001C0804100C181400080
:10245500C1814001C0804100C1814001C08041016E
:10246500C0804100C1814000C1814001C08041015F
:10247500C0804100C1814001C0804100C181400050
:10248500C1814001C0804101C0804100C18140003F
:10249500C1814001C0804100C1814001C08041012E
:1024A500C0804100C1814000C1814001C08041011F
:1024B500C0804100C1814001C0804100C181400010
:1024C500C1814001C0804100C1814001C0804101FE
:1024D500C0804100C1814001C0804100C1814000F0
:1024E500C1814001C0804101C0804100C1814000DF
:1024F500C1814001C0804100C1814001C0804101CE
:10250500C0804100C1814000C0C101C30302C2C6F1
:102515000607C705C5C404CC0C0DCD0FCFCE0E0ADA
:10252500CACB0BC90908C8D81819D91BDBDA1A1E7A
:10253500DEDF1FDD1D1CDC14D4D515D71716D6D24A
:102545001213D311D1D010F03031F133F3F232360A
:10255500F6F737F53534F43CFCFD3DFF3F3EFEFA1A
:102565003A3BFB39F9F83828E8E929EB2B2AEAEE5A
:102575002E2FEF2DEDEC2CE42425E527E7E626228A
:10258500E2E323E12120E0A06061A163A3A26266EA
:10259500A6A767A56564A46CACAD6DAF6F6EAEAA5A
:1025A5006A6BAB69A9A86878B8B979BB7B7ABABEFA
:1025B5007E7FBF7DBDBC7CB47475B577B7B67672CA
:1025C500B2B373B17170B0509091519353529296CA
:1025D500565797559594549C5C5D9D5F9F9E5E5A9A
:1025E5009A9B5B99595898884849894B8B8A4A4EDA
:1025F5008E8F4F8D4D4C8C4484854587474686820A
:10260500424383418180403C6D303D000000003CE9
:102615006D313D000000003C6D323D000000003C86
:102625006D333D000000003C6D343D000000003C72
:102635006D353D000000003C6D363D000000003C5E
:102645006D373D000000003C6D383D000000003C4A
:102655006D393D000000003C6D31303D0000003C0F
:102665006D31313D0000003C6D31323D0000003CD4
:102675006D31333D0000003C6D31343D0000003CC0
:072685006D31353D0000003E
:0100210022BC
:030023000244FA9A
:0B44FA00C0E0C083C082C0D075D018A5
:10450500309827E5E92464F5EB30D707E5F904F59C
:10451500FB800385F9FBD29174752539F582E43466
:104525006AF583E599F00539C298309931E53EC3BE
:104535009538501BAF3E053E74752FF582E4346BFC
:10454500F583E0FF521FA2D0B3929B8F99800DE5B2
:0E4555003EC395384006053ED296C290C299EC
:09456300D0D0D082D083D0E03228
:10337D007BFF7A2179B51226EE90688FE070147577
:10338D0059FF755A22755B0C7BFF7A2179CE122677
:10339D00EE80127559FF755A22755B1B7BFF7A21E2
:1033AD0079CE1226EE7BFF7A22792A1226EE7BFF4A
:1033BD007A227959A21DE433F5591226EE75590179
:1033CD00755A6A755B2B7BFF7A22797C1226EE90FB
:1033DD006B97E0FEA3E0FFC3E49FFFE49EFEAB0707
:1033ED00FA3395E0F9F87F007E8C7D0A7C00122B74
:1033FD00178F5C8E5B8D5A8C597BFF7A22799612D2
:10340D0026EE7BFF7A2279CCA219E433F5591226E8
:10341D00EE7BFF7A2279EF906890E0F5591226EE57
:10342D00E4906BA9F0906BA9E0FFC3648094904089
:10343D00030234CF9069DA7420F0E4A3F0EF3395F2
:10344D00E0FEEF7803C333CE33CED8F9240CF582EA
:10345D0074263EAF82FE1240FFEF4E6041E4906B4A
:10346D00ABF01248A3906BAAEFF0643C601BE0FF39
:10347D00A3E0FE04F0EEFD3395E0FC74DA2DF58249
:10348D0074693CF583EFF080D9906BABE0FF339519
:10349D00E0FE74DA2FF58274693EF583E4F0906BEB
:1034AD00A9E0F559755A01755B69755CDA04F55D2E
:1034BD007BFF7A2379131226EE906BA9E004F002BC
:1034CD003432906B95E0FEA3E0FF7C007D0A122A5A
:0E34DD00378E598F5A7BFF7A23793E1226EEE6
:0134EB0022BE
:06472C00AC05AB07AA0674
:104732009069D974FFF0906A2AF0AF041CEF602DE3
:104742000BEBAE0270010A14F5828E83E0FF9069D2
:10475200D9E06FFF90240C93FE906A2AE06E906974
:0D476200D9F0EF90250C93906A2AF080CDDD
:01476F002227
:04430800A907AE0350
:10430C00E4906BA9F0906BA9E0FFC39440501B851F
:10431C004482854383A3E5822FF582E43583F583BC
:10432C00E4F0906BA9E004F080DB85448285438344
:10433C007406F0A3E9F0854482854383A3A3740833
:10434C00F0EED39401400E854482854383A3A3A34E
:10435C007416F0800C854482854383A3A3A3741444
:10436C00F0E5442404F582E43543F583EDF0E544AF
:0B437C00241CF582E43543F583EEF0CD
:014387002213
:1008A4007E237F5D1240FFEF4E70037F0122E490B0
:1008B400688FF07E237F601240FFEF4E601B12486A
:1008C400A38F51E551B4310690688F740AF0E55155
:1008D400B4320690688F7464F07E237F661240FF02
:1008E400EF4E60351248A3906A2BEFF01248A390A4
:1008F4006A2CEFF01248A3906A2DEFF01248A390EF
:100904006A2EEFF01248A3906A2FEFF01248A390DA
:100914006A30EFF0E4A3F08013906A2B7431F0A3F3
:10092400F0A3F0A3F0A3F0A3F0E4A3F07E237F6C84
:100934001240FFEF4E602312462FA804A905AA0611
:10094400AB077F007E8C7D0A7C00122B17122BA92B
:10095400906B97EEF0A3EFF0800A906B9774FFF022
:10096400A374B8F07E237F721240FFEF4E600A1228
:10097400462F906890EFF08005E4906890F07E2315
:100984007F781240FFEF4E601612462FE47B0AFA7E
:10099400F9F8122A8C906B95EEF0A3EFF0800A9090
:1009A4006B957403F0A374E8F07E237F7E1240FFFE
:1009B400EF4E600D12462FEC4D4E4F24FF921D80DA
:1009C40002C21D7E237F841240FFEF4E600C12484A
:1009D400A3EF24D024FF92198002C219E4F543F551
:1009E40044301D5F854482854383A374FEF08544AF
:1009F40082854383A3A37403F0854482854383A340
:100A0400A3A37408F0E5442401FFE43543FE7D0309
:100A140012472C9069D9E0FFE5442404F582E435BB
:100A240043F583EFF0906A2AE0FFE5442405F5825C
:100A3400E43543F583EFF08544828543837405F000
:100A4400020ADB854482854383A374FEF0854482D5
:100A5400854383A3A37403F0854482854383A3A3BE
:100A6400A37408F0E5442404F582E43543F5837463
:100A740055F0E5442405F582E43543F58374AAF082
:100A8400E5442406F582E43543F5837433F0E54404
:100A94002407F582E43543F58374CCF0E54424015E
:100AA400FFE43543FE7D0712472C9069D9E0FFE54A
:100AB400442408F582E43543F583EFF0906A2AE094
:100AC400FFE5442409F582E43543F583EFF08544DA
:100AD400828543837409F074202544F544E4354346
:100AE400F543854482F583E4F09069D804F0E4F595
:100AF40051AF51EF3395E0FEEF7803C333CE33CEDD
:100B0400D8F9240CF58274263EAF82FE1240FFEF22
:100B14004E7003020FF412462F8F4AE54A70030207
:100B24001002E54AB4FF03E4F54A201D03020BFD5D
:100B3400854482854383A3E54AF0854482854383C3
:100B4400A3A37401F0854482854383A3A3A3F090F7
:100B54006A2BE0FFE5442404F582E43543F583EF92
:100B6400F0906A2CE0FFE5442405F582E43543F572
:100B740083EFF0906A2DE0FFE5442406F582E43526
:100B840043F583EFF0906A2EE0FFE5442407F582F5
:100B9400E43543F583EFF0906A2FE0FFE544240841
:100BA400F582E43543F583EFF0906A30E0FFE544E5
:100BB4002409F582E43543F583EFF0E5442401FF8D
:100BC400E43543FE7D0912472C9069D9E0FFE544E2
:100BD400240AF582E43543F583EFF0906A2AE0FFB6
:100BE400E544240BF582E43543F583EFF085448234
:100BF400854383740BF0020CB5854482854383A33B
:100C0400E54AF0854482854383A3A37401F0906A86
:100C14002BE0854482854383A3A3A3F0906A2CE050
:100C2400FFE5442404F582E43543F583EFF0906A4C
:100C34002DE0FFE5442405F582E43543F583EFF028
:100C4400906A2EE0FFE5442406F582E43543F583FB
:100C5400EFF0906A2FE0FFE5442407F582E4354382
:100C6400F583EFF0906A30E0FFE5442408F582E470
:100C74003543F583EFF0E5442401FFE43543FE7D7D
:100C84000812472C9069D9E0FFE5442409F582E471
:100C94003543F583EFF0906A2AE0FFE544240AF532
:100CA40082E43543F583EFF0854482854383740AF7
:100CB400F0E544241CF582E43543F583E4F0742024
:100CC4002544F544E43543F5439069D8E004F085C0
:100CD4004482854383E4F01248A3EF122C180DC715
:100CE400000DC7210D28230FE22A0FB92F0D473B12
:100CF4000DC73C0FB93E0EC2430ECE450E74460ED0
:100D0400A7490E9B4C0E50500E5C510FD0520E68EA
:100D1400530E80550F35610F61620F8D630F0B7396
:100D240000000CDB1248A375F008EFA42484F582BC
:100D3400E5F03424AF82FE1240FFEF4E6099124674
:100D44002F8094E5442401FFE43543FE7D041247DB
:100D54002C9069D9E0FFE5442405F582E43543F598
:100D640083EFF0906A2AE0FFE5442406F582E43537
:100D740043F583EFF0E5442401FFE43543FE7D06AB
:100D840012472C9069D9E0FFE5442407F582E43545
:100D940043F583EFF0906A2AE0FFE5442408F582E6
:100DA400E43543F583EFF074202544F544E43543FA
:100DB400F5439069D8E004F0854482854383E4F0E8
:100DC400020CDB854482854383E06075E54424019D
:100DD400FFE43543FE7D0412472C9069D9E0FFE51A
:100DE400442405F582E43543F583EFF0906A2AE064
:100DF400FFE5442406F582E43543F583EFF0E5444A
:100E04002401FFE43543FE7D0612472C9069D9E0A6
:100E1400FFE5442407F582E43543F583EFF0906A57
:100E24002AE0FFE5442408F582E43543F583EFF036
:100E340074202544F544E43543F5439069D8E0042F
:100E4400F0854482854383E4F0020FF47B0FE4FDD4
:100E5400AF4A124308020CDB7B0F7D04AF4A1243F6
:100E640008020CDB7B0F7D08AF4A124308020CDB3F
:100E74007B017D40AF4A124308020CDB301D0C7B22
:100E84000E7D11AF4A124308020CDB7B0E7D10AFBE
:100E94004A124308020CDB7B0E7D14AF4A1243084E
:100EA400020CDB301D0C7B0E7D21AF4A124308027D
:100EB4000CDB7B0E7D20AF4A124308020CDB7B0F58
:100EC4007D30AF4A124308020CDB7B017D0FAF4A31
:100ED400124308854482854383A3A37405F08544A3
:100EE40082854383A3A3A3E4F0E5442404F582E4C8
:100EF4003543F583E4F0E544241CF582E43543F5F9
:100F040083740FF0020CDB854482854383A3A3A37F
:100F14007411F0E5442404F582E43543F583E0F0EC
:100F2400E544241CF582E43543F5837401F0020C96
:100F3400DB854482854383A3A3A37411F0E5442491
:100F440004F582E43543F583E04401F0E544241CD0
:100F5400F582E43543F5837401F0020CDB854482A9
:100F6400854383A3A3A37411F0E5442404F582E428
:100F74003543F583E04402F0E544241CF582E4356E
:100F840043F5837401F0020CDB854482854383A31B
:100F9400A3A37411F0E5442404F582E43543F583F6
:100FA400E04403F0E544241CF582E43543F58374FE
:100FB40001F0020CDB1248A3EF24D0FFE544241D0A
:100FC400F582E43543F583EFF0020CDBE544241E9F
:100FD400F582E43543F583E04401F0020CDBE5449B
:100FE400241EF582E43543F583E04402F0020CDB71
:100FF4000551C3E551648094905003020AF5E4F569
:1010040043F544FFF551854482854383E0607CA326
:10101400A3E064087034E544241FF582E43543F505
:1010240083E551F0E544241CF582E43543F583E07F
:10103400FEB401020551EEB40F0674042551F551B6
:10104400EEB40E0674032551F5518544828543831D
:10105400A3A3E064057026E544241FF582E4354328
:10106400F583EFF0E544241CF582E43543F583E091
:10107400FEB401010FEEB40F0474042FFF74202595
:1010840044F544E43543F54302100AE4F543F544DA
:01109400FF5C
:011095002238
:1047DC00C2A9438902758C48758A4875D90475DB62
:1047EC004875DC4875DD4875DE48E4F5E9F5F9C235
:0647FC00D9D28CD2DE22AE
:103FE10043AB01C2E8C2EAE4FFEFC454F0F5B1C348
:103FF100EF64809488500575B3D08003E4F5B3EF86
:104001007026F5B275BC01F5BDF5BEF5BF75C4FFEF
:10401100F5C5F5C6F5C7F5A3F5A3F5A3F5A3F5A376
:10402100F5A3F5A3F5A38027E4F5B275BCC8F5BDEA
:10403100F5BE75BF7875C4FFF5C5F5C675C778F5CA
:10404100A3F5A3F5A3F5A3F5A3F5A3F5A3F5A30F95
:10405100BF0E9690688FE0FF25E0F5B475B50C753D
:10406100B66C75A11275AB0275C13E75C3FF75C201
:01407100034B
:01407200222B
:1045CF0075B180E4F5B3F5B28527BCE5285403FF38
:1045DF0033333354F8FFE52854E04FFFE529C41374
:1045EF0054074FF5BDE52933333354F8FFE52AC49B
:1045FF001354074FF5BEE52A33333354F8F5BF850F
:10460F002CA3852DA3852EA3852FA38530A38531BC
:10461F00A38532A38533A3E52B540F2450F5B32282
:10377700E59B541F6020200B1A7E237F8A1239880D
:10378700E59B541FFF7E007D03123A897E237F94B9
:10379700123988E4F59BE5BA30E008E4F5B375B172
:1037A70080F5B2E5CFF47003023881755301E4F573
:1037B70052E5CFF45553700302386FE552C454F005
:1037C700F5B1E5B2547F6420706FE5B3540FF52B64
:1037D70085BC27E5BD541FFF131313541FFFE5BD19
:1037E70054E044184FF528E5BDC43354E0FFE5BE67
:1037F700131313541F4FF529E5BEC43354E0FFE5F7
:10380700BF131313541F4FF52A85A32C85A32D85AA
:10381700A32E85A32F85A33085A33185A33285A346
:1038270033E4F5B2E527547EB5270575B350800319
:1038370075B3D0E52B2405FF22E5B2549F60232002
:103847000B207E237F97123988AFB27E007D03124B
:103857003A89AFB37E007D03123A897E237FA21295
:103867003988E4F5B275B3D0E55325E0F553055231
:0C387700E552C3940850030237B87F00EC
:013883002222
:103EA700C21AE4F539F50BD296F538F53EF525FF3C
:103EB70074352FF582E4346AF583E4F074932FF5B3
:103EC70082E43468F583E4F00FBF40E4E49069D6F8
:103ED700F0A3F0F53FF54F1208A4123FE1C2ADE49D
:103EE700F5C9D2CDD2CCC2C9C2CAF5CDF5CC906B3B
:103EF70097E0F5CBA3E0F5CA85CBCD85CACCE4F531
:103F0700985387BF301906D29FD29E8002D29E4314
:103F17008740C29FC2ACC298C29975B81075B710D6
:103F2700D2CAD29CD2AC1247DCC2D9E5E92464F5E7
:0D3F3700EB30D706E5F904F5FB2285F9FB18
:013F4400225A
:0100220022BB
:0148F10022A4
:0148F20022A3
:10484A0090637CE0B40118906384E0F5459063833B
:10485A00E0F546906382E0F547906381E0F54822EF
:10307000854482854383E07010F543F5448544829E
:10308000854383E070037F0122854482854383A3C7
:10309000A3E064017060753501854336854437E5EA
:1030A00044241CF582E43543F583E0601674202542
:1030B00044F544E43543F543854482F583E070B03C
:1030C0007F0122E5442401FFE43543F5838F8263C9
:1030D000A201906B7563A2017F0C122DBE85448204
:1030E000854383E0F538300B030231E77E237FA46C
:1030F0001239880231E7854482854383A3A3E0FF28
:1031000064036003EF703F052553250FE49069D6F3
:10311000F0A3F0E5442401FFE43543F5838F826397
:10312000A201906B7563A2017F0C122DBE854482B3
:10313000854383E0F538300B030231E77E237FAE11
:103140001239880231E7AB35AA36A93790001C1234
:1031500029E8700E74202544F544E43543F5430214
:103160003070E544241EF582E43543F583E030E118
:1031700012E525600E74202544F544E43543F543FB
:10318000023070854482854383A3E0906B75F0859F
:103190004482854383A3A3E0906B76F085448285C7
:1031A0004383A3A3A3E0906B77F0E5442404F58266
:1031B000E43543F583E0906B78F0E5442405F5822F
:1031C000E43543F583E0906B79F0E5442406F5821D
:1031D000E43543F583E0906B7AF0753806200B07F1
:1031E0007E237FB4123988E4F53ED290C291C29614
:1031F000C2992099FDD299200B0B7E6B7F75E4FB61
:07320000AD38123B837F0093
:0132070022A4
:10365200E54FC394404003E4F54FE534C394404042
:1036620003E4F53474932534F582E43468F583E099
:10367200FF30E17B74932534F582E43468F583EFFF
:1036820054FDF0E4906478F0A3740DF090667CE051
:1036920090647AF0A37419F0A37444F0A37439F01F
:1036A200E534C4135407FF906890E02F90647EF0D5
:1036B200E534541F04A3F0A37408F0E53425E02593
:1036C200E024D6F582E43468F58363A20190648134
:1036D20063A2017F04122DBE906485E548F0A3E544
:1036E20047F0A3E546F0A3E545F005347F012274D7
:1036F20035254FF582E4346AF583E0FF30E16F74DB
:1037020035254FF582E4346AF583EF54FDF0E490F9
:103712006478F0A3740DF090667CE090647AF0A374
:103722007419F0A37448F0A37479F0E54F131313DE
:10373200541FFF906890E02F90647EF0E54F54078D
:1037420025E025E02480A3F0A37408F0F5F0E54F0E
:10375200A4248FF582E5F03466F58363A2019064B8
:103762008163A2017F08122DBE054F7F0122054F02
:0537720005347F002278
:0148F30022A2
:1016DE007435253FF582E4346AF583E020E0020597
:1016EE003FE53FC394404003E4F53F74932524F552
:1016FE0082E43468F583E020E0020524E524C394F7
:10170E00404003E4F524123777EF7003021801E529
:10171E0027B4010C852F45852E46852D47852C48EF
:10172E00E52A640F6003021801906890E0FF6529B6
:10173E00600302180174932524F582E43468F5835E
:10174E00E0FE30E05174932524F582E43468F5838D
:10175E00EE54FEF0752744752839E524C41354075A
:10176E00FEEF2EF529E524541F04F52A752B08E506
:10177E002425E025E024D6F582E43468F5837D2C1B
:10178E007F04122DB5854830854731854632854513
:10179E00331245CF805D7435253FF582E4346AF50A
:1017AE0083E0FF30E04D7435253FF582E4346AF571
:1017BE0083EF54FEF0752748752879E53F13131310
:1017CE00541FFF906890E02FF529E53F540725E060
:1017DE0025E02480F52A752B0875F008E53FA42432
:1017EE008FF582E5F03466F5837D2C7F08122DB5DA
:1017FE001245CF2002030218BFC2020549E549C3B4
:10180E0094644066E4F549AF48AE47AD46AC45FA40
:10181E00F9F8EF2401F548EA3EF547E93DF546E8CB
:10182E003CF545E47B3CAF48AE47AD46AC45122B8C
:10183E0017AC00AD01AE02AF03E4FBFAF9F8C31228
:10184E002BB77026F55174932551F582E43468F563
:10185E0083E030E20E74932551F582E43468F5830B
:10186E007403F00551E551B440DC906892E004F049
:10187E007006906891E004F0D3906892E094B8906E
:10188E006891E0940B402AE4F0A3F0F551743525ED
:10189E0051F582E4346AF583E030E20E7435255159
:1018AE00F582E4346AF5837403F00551E551B440D2
:1018BE00DC20D903021CABC2D9E539D39400500306
:1018CE00021C1DC291853942E4F539F50B7E6A7F03
:1018DE0075AD4212472C200B127E237FBD12398824
:1018EE007E6A7F75E4FBAD42123B83906A2AE0FF6D
:1018FE009069D9E04F6010300B03021C1D7E237FD0
:10190E00C4123988021C1D854482854383A3E0FFDF
:10191E00906A75E06F6010300B03021C1D7E237FF2
:10192E00D0123988021C1D854482854383A3A3E00F
:10193E006401703D906A76E0601A200B077E237F6B
:10194E00DF123988E544241CF582E43543F583E43F
:10195E00F0021C1DD21B200B077E237FF712398845
:10196E00E544241CF582E43543F5837401F0021C32
:10197E001DD21BE542C39406501DAB35AA36A937BE
:10198E0090001CE4122A15300B03021C1D7E237FCF
:10199E00FD123988021C1DE544241FF582E43543EF
:1019AE00F583E075F002A4FF9069D6E5F0F0A3EFA1
:1019BE00F0E4F551E544241CF582E43543F583E06B
:1019CE00FD7C0074017E00A851088005C333CE3320
:1019DE00CED8F9FFEE5CFEEF5D4E7003021C128551
:1019EE004482854383A3A3E064086003021B28F5A9
:1019FE003AE55175F003A42476F582E4346AF58352
:101A0E00E0543FF53BE55175F003A42477F582E4ED
:101A1E00346AF583E0F53CE55175F003A42478F5BE
:101A2E0082E4346AF583E0F53DAF3DAE3CAD3BACB0
:101A3E003AE544241DF582E43543F583E0F9F812C6
:101A4E002BC88F3D8E3C8D3B8C3AE544241EF5828F
:101A5E00E43543F583E030E026E55175F003A42428
:101A6E0076F582E4346AF583E030E713AF3DAE3CA1
:101A7E00AD3BAC3A122BA98F3D8E3C8D3B8C3A90F0
:101A8E0069D6E0FEA3E0248FF58274663EF583E00E
:101A9E00653D60299069D6E0A3E0FF248FF582743E
:101AAE00663EF583E53DF0EF7803CEC313CE13D833
:101ABE00F92435F582746A3EF5837407F09069D780
:101ACE00E004F070069069D6E004F09069D6E0FE6E
:101ADE00A3E0248FF58274663EF583E0653C6029B1
:101AEE009069D6E0A3E0FF248FF58274663EF583FD
:101AFE00E53CF0EF7803CEC313CE13D8F92435F5B9
:101B0E0082746A3EF5837407F09069D7E004F07032
:101B1E00069069D6E004F0021C12E544241FF582FB
:101B2E00E43543F583E075F004A4FDACF0E55175A2
:101B3E00F004A42DFEEC35F09069D6F0A3CEF0E5BE
:101B4E005125E025E02479F582E4346AF583E0FF3F
:101B5E009069D7E024D6F582E43468F583EFF090EF
:101B6E0069D7E004F070069069D6E004F0E55125DF
:101B7E00E025E02478F582E4346AF583E0FF90698D
:101B8E00D7E024D6F582E43468F583EFF09069D778
:101B9E00E004F070069069D6E004F0E55125E025EA
:101BAE00E02477F582E4346AF583E0FF9069D7E0AC
:101BBE0024D6F582E43468F583EFF09069D7E0041B
:101BCE00F070069069D6E004F0E55125E025E0249A
:101BDE0076F582E4346AF583E0FF9069D7E024D687
:101BEE00F582E43468F583EFF0E544241FF582E4D2
:101BFE003543F583E025512493F582E43468F5836B
:101C0E00E04404F00551E551640460030219C290EA
:101C1E006B95E0FEA3E0FF4E6020201C1BE025E943
:101C2E00F5EB30D708EE25F904F5FB8008906B959F
:101C3E00E025F9F5FBD21C22C21C201B0DAB35AAE8
:101C4E0036A93790001CE4122A15E538600B742073
:101C5E002544F544E43543F543E5E924E8F5EB3056
:101C6E00D708E5F92404F5FB8006E5F92403F5FB16
:101C7E00123070EF7027854482854383A3A3E0B4AE
:101C8E000319E5E924F4F5EB30D708E5F92402F55C
:0D1C9E00FB8005E5F904F5FBD21B22C21BFB
:011CAB002216
:03001E007F00223E
:10407F00021096E493A3F8E493A34003F68001F2B1
:10408F0008DFF48029E493A3F85407240CC8C33342
:10409F00C4540F4420C8834004F456800146F6DF11
:1040AF00E4800B01020408102040809048EAE47E6F
:1040BF00019360BCA3FF543F30E509541FFEE49306
:1040CF00A360010ECF54C025E060A840B8E493A3CD
:1040DF00FAE493A3F8E493A3C8C582C8CAC583CAF8
:1040EF00F0A3C8C582C8CAC583CADFE9DEE780BEB0
:0148F00000C7
:1029E800BB010CE58229F582E5833AF583E02250A4
:1029F80006E92582F8E622BBFE06E92582F8E222EE
:0D2A0800E58229F582E5833AF583E4932207
:102A1500F8BB010DE58229F582E5833AF583E8F0F7
:102A2500225006E92582C8F622BBFE05E92582C8A3
:022A3500F2228B
:102A3700BC000BBE0029EF8DF084FFADF022E4CC83
:102A4700F875F008EF2FFFEE33FEEC33FCEE9DEC4C
:102A5700984005FCEE9DFE0FD5F0E9E4CEFD22ED92
:102A6700F8F5F0EE8420D21CFEADF075F008EF2FDC
:102A7700FFED33FD4007985006D5F0F222C398FDCD
:052A87000FD5F0EA226A
:102A8C00E88FF0A4CC8BF0A42CFCE98EF0A42CFCE9
:102A9C008AF0EDA42CFCEA8EF0A4CDA8F08BF0A467
:102AAC002DCC3825F0FDE98FF0A42CCD35F0FCEBC6
:102ABC008EF0A4FEA9F0EB8FF0A4CFC5F02ECD398B
:0F2ACC00FEE43CFCEAA42DCE35F0FDE43CFC22F8
:102ADB0075F008758200EF2FFFEE33FECD33CDCCB2
:102AEB0033CCC58233C5829BED9AEC99E582984035
:102AFB000CF582EE9BFEED9AFDEC99FC0FD5F0D612
:102B0B00E4CEFBE4CDFAE4CCF9A88222B800C1B93B
:102B1B000059BA002DEC8BF084CFCECDFCE5F0CB79
:102B2B00F97818EF2FFFEE33FEED33FDEC33FCEBB2
:102B3B0033FB10D703994004EB99FB0FD8E5E4F96D
:102B4B00FA227818EF2FFFEE33FEED33FDEC33FC5A
:102B5B00C933C910D7059BE99A4007EC9BFCE99A4E
:102B6B00F90FD8E0E4C9FAE4CCFB2275F010EF2F93
:102B7B00FFEE33FEED33FDCC33CCC833C810D70793
:102B8B009BEC9AE899400AED9BFDEC9AFCE899F8CE
:0E2B9B000FD5F0DAE4CDFBE4CCFAE4C8F92261
:0E2BA900C3E49FFFE49EFEE49DFDE49CFC223D
:102BB700EB9FF5F0EA9E42F0E99D42F0E89C45F074
:012BC70022EB
:102BC800E8600FECC313FCED13FDEE13FEEF13FFEB
:032BD800D8F1220F
:0C2BDB00ECF0A3EDF0A3EEF0A3EFF0226D
:102BE700A8828583F0D083D082122BFE122BFE128F
:102BF7002BFE122BFEE473E493A3C583C5F0C583B4
:102C0700C8C582C8F0A3C583C5F0C583C8C582C837
:012C1700229A
:102C1800D083D082F8E4937012740193700DA3A34B
:102C280093F8740193F5828883E47374029368605F
:062C3800EFA3A3A380DF5F
:10268C00E5652459F8E60565227856301702785925
:10269C00E475F001122C69022C3E2010EB7F2ED237
:1026AC00108018EF540F2490D43440D4FF30140B06
:1026BC00EF24BFB41A0050032461FFE566600215D5
:1026CC00660569E5697002056830170D7856E47582
:1026DC00F001122C69EF022C570246E57403D21755
:1026EC008003E4C217F5658B568A578958E4F56662
:1026FC00F568F569E56660077F201226C780F575D9
:10270C0067FFC211C210C212C213C215C216C21880
:10271C00122695FF700D3017057F001226D8AF6971
:10272C00AE6822B4255FC2D5C214122695FF24D000
:10273C00B40A00501A75F00A786630D50508B6FF51
:10274C000106C6A426F620D5047002D21380D92423
:10275C00CFB41A00EF5004C2E5D2140228D8D2111B
:10276C0080C6D21080C0D21280BCD2D580BAD2150D
:10277C0080B47F201226C72012077401B566004072
:10278C00F112268CFF1226C7022700D218D216800F
:10279C009512268CFB12268CFA12268CF94A4B7059
:1027AC000679A97A297BFF20122EE566602A7E0025
:1027BC008E827583001229E860060EEE656770F054
:1027CC00C2D5EBC0E0EAC0E0E9C0E0EE12291FD0B0
:1027DC00E0F9D0E0FAD0E0FB122C3EFF60AAEBC08F
:1027EC00E0EAC0E0E9C0E01226C7D0E02401F9D04D
:1027FC00E03400FAD0E0FBE5670460DCD567D980F3
:10280C00877BFF7A29791BD212809C791080027900
:10281C0008C216C2188008D2D5790A8004790AC277
:10282C00D5E567047002F567E4FAFDFEFF12268C0D
:10283C00FC7B0820111312268CFD7B1030100A1221
:10284C00268CFE12268CFF7B20EC3382D592D55041
:10285C0013C3E43010069FFFE49EFEE42011039D99
:10286C00FDE49CFCE4CBF8C211EC700CCFCECDCCCB
:10287C00E824F8F870F38017C3EF33FFEE33FEED66
:10288C0033FDEC33FCEB33FB994002FB0FD8E9EB47
:10289C00301105F8D0E0C448B211C0E00AEC4D4E3E
:1028AC004F78207B0070C2EAB5670040BCC0E012D4
:1028BC002921D0F0D0E0201104C4C0E0C4B211C072
:1028CC00F01226B0D0F0D5F0EB022700122C18270E
:1028DC009D53281758276E4C276A42281B4F2823D4
:0F28EC0044282349278343282955280D46280DC2
:1028FB0045280D4729C95027722D27762E27992B4E
:10290B00277A2327972029B22A27324800002791BC
:10291B003F3F3F00790AA2D5201314301509B91097
:10292B00020404B9080104A2D520160250010420A8
:10293B0012689212B566005034C0E07F2030131934
:10294B007F30A21272167215500F122978C212C262
:10295B0016C215C2187F30800F301503E9C0E01284
:10296B0026C7301503D0E0F9D0E0B566CC3015178B
:10297B007F30B9100C1226C77F583014077F788030
:10298B0003B908031226C73012057F2D0226C77F15
:10299B00202018F87F2B2016F322921280CF286E5E
:1029AB00756C6C2900D21112268C3011F8C211787B
:1029BB006630D50108F60227322D504349581226AE
:1029CB008C2403B405004001E49029C4931226B86B
:0D29DB00743A1226B8D2137566040228174C
:102ECC008B568A578958E4F562F561F560F55FF524
:102EDC005DF55EE55A455B45596012EBC0E0EAC012
:102EEC00E0E9C0E0AB59AA5AA95B122C79AB5605A4
:102EFC0058E558AA577002055714F9122C3EF56381
:102F0C00C394094007E563D3940D40E1E563642065
:102F1C0060DBE563B42D05435E038016E563B42BDB
:102F2C0005435E01800C74FF2558F55874FF355726
:102F3C00F557E55C60046410703FAB56AA57A9586E
:102F4C00122C3E64306009E55C702E755C0A802999
:102F5C009000011229E8FF64786004EFB458134321
:102F6C005E01755C1074022558F558E43557F55719
:102F7C008007E55C7003755C08AB560558E558AAEC
:102F8C00577002055714F9122C3EF563C394614037
:102F9C000AE563D3947A50035363DF74D02563F549
:102FAC0063C3940A400CE5639411406D74F9256376
:102FBC00F563E563D3955C5060435E01856267857C
:102FCC006166856065855F64AF5C7E00E4FCFDAB8B
:102FDC0062AA61A960A85F122A8CC8ECC8C9EDC9A5
:102FEC00CAEECACBEFCBE4FCFDFEEB2563F562EE3B
:102FFC003AF561ED39F560EC38F55FAF62AE61AD75
:10300C0060FCAB67AA66A965A864D3122BB7500302
:10301C00022F85435E04022F85E55E20E003E480E9
:10302C002DE55A455B4559601EAB56E55824FFF912
:10303C00E55734FFFAEBC0E0EAC0E0E9C0E0AB5979
:10304C00AA5AA95B122C79E55E30E20774FFFFFEE9
:10305C00FDFC22E55EAF62AE61AD60AC5F30E103BA
:04306C00022BA92268
:102C3E00BB010689828A83E0225002E722BBFE0294
:092C4E00E32289828A83E49322C7
:102C5700BB010689828A83F0225002F722BBFE015C
:022C6700F32256
:102C6900FAE6FB0808E6F925F0F618E6CA3AF6226C
:102C7900BB011A89828A83D0F0D0E0F8D0E0F9D07C
:102C8900E0FAD0E0FBE8C0E0C0F0022CD15016E930
:102C9900F8D083D082D0E0F9D0E0FAD0E0FBC0824E
:102CA900C083022CC8BBFE16E9F8D083D082D0E0DD
:0F2CB900F9D0E0FAD0E0FBC082C083022CDA220F
:092CC800EBF608EAF608E9F62231
:092CD100EBF0A3EAF0A3E9F02204
:092CDA00EBF208EAF208E9F2222B
:00000001FF
